:10000000000011298207303431343234333434342F
:100010003534363437343834393482072D343D346E
:1000200050344D34453454342B34DF344334820758
:10003000A034ED344734493446344E344F344334DD
:10004000A0342E34473445345234EC348207A03483
:10005000A034E034653464346F344D34A0346E34ED
:1000600077346F34643474347534683453348207AD
:10007000A034A034E034653464346F344D34A0349B
:100080006C3461346D3472346F344E34A034A03427
:100090008207A034E034653464346F344D34A034C6
:1000A0002E3470346D346F3443348207A034E0341E
:1000B000653464346F344D34A0342E3474346E346B
:1000C0004934A0348207A034A034A034E03477341B
:1000D0006F344C34A03479347434693472346134FC
:1000E0006C346F345034A0345234543450344D3462
:1000F00043342F3454344E3449348207A034A0346E
:10010000E0346834673469344834A0347934743462
:100110006934723461346C346F345034A0345234E6
:10012000543450344D3443342F3454344E344934E1
:100130008207A034E0343134A0346534753465343A
:1001400075345134A03474346C34753461344634AD
:100150008207A034E0343234A03465347534653419
:1001600075345134A03474346C347534613446348D
:100170008207A034E0343434A034653475346534F7
:1001800075345134A03474346C347534613446346D
:100190008207A034E0343634A034653475346534D5
:1001A00075345134A03474346C347534613446344D
:1001B0008207A0343D347434653473345434A0342D
:1001C000ED347434653473345434A0342E344734ED
:1001D00045345234EC348207A0343D3473347934DE
:1001E00068345434A034ED3473347934683454347E
:1001F000A0342E34473445345234EC348207A034D2
:100200003D3450344D3445345434A034ED345034FE
:100210004D3445345434A0342E34473445345234AC
:10022000EC340000831203131F108316031387306E
:10023000810083120313850186018701831603134E
:1002400086309F0083160313013085008316031345
:100250003F30860083160313003087008312031398
:1002600000308B00BF01BD0102243A21DE2321238F
:100270007E233329061E3A29FF221F3087000723D9
:10028000FF221630870007230D30B800FF2203013C
:10029000831203133808172087000723B80B462959
:1002A000A7226429FF22831203130B308700072340
:1002B0000D30B800FF220301831203133808172002
:1002C00087000723B80B5A293A1891213A1C9E211E
:1002D000BA18AB21BA1CB821A2223A19D2213A1D70
:1002E000C521BA1D78293A1A06223A1EEC217C292A
:1002F0003A1AF9213A1EDF21061C1322861C1B2202
:10030000061D2322861D2B22061A5229FF221F308A
:10031000870007235322061A8B29061E8D29BA014E
:1003200008000F30B800FF220301831203133808BE
:10033000262087000723B80B932908000F30B80048
:10034000FF22030183120313380837208700072395
:10035000B80BA02908000B30B800FF22030183125C
:1003600003133808552087000723B80BAD29080070
:100370000B30B800FF220301831203133808482012
:1003800087000723B80BBA2908001930B800FF22EC
:100390000301831203133808622087000723B80B78
:1003A000C72908001930B800FF2203018312031384
:1003B00038087D2087000723B80BD42908000E30A9
:1003C000B800FF2203018312031338089820870026
:1003D0000723B80BE12908000E30B800FF22030103
:1003E000831203133808A82087000723B80BEE29CF
:1003F00008000E30B800FF220301831203133808EF
:10040000B82087000723B80BFB2908000E30B8007E
:10041000FF220301831203133808C8208700072333
:10042000B80B082A0800061C132A3A18192A3A148D
:100430001A2A3A100800861C1B2ABA18212ABA1454
:10044000222ABA100800061D232A3A19292A3A1529
:100450002A2A3A110800861D2B2AB8013A08B8004A
:10046000B80CB80C3810B8113812B8123813B813C9
:10047000023083013802031D402ABA113A16522A6B
:10048000043083013802031D482ABA153A16522A4D
:10049000063083013802031D502ABA113A12522A3B
:1004A000BA153A12080083120313BA133A13BA1298
:1004B000E522992287229922831203138C01831249
:1004C0000313903093008C1D632A83160313111BB2
:1004D000862A9922831203138C01013093008C1D0C
:1004E0006F2A83160313111B862A99228312031382
:1004F0008C01831203133A0893008C1D7D2A831606
:100500000313111B862A99229322F62208008316D0
:1005100003131114941D8A2A0800831603139114DF
:10052000941D902A0800831603131115141E962A91
:1005300008008316031314199B2A11081F39031D81
:100540009D2A0800FF220C30870007230800E522BF
:10055000992287229922831203138C0190309300F1
:100560008C1DB02A83160313111BE12A99228312D2
:1005700003138C01013093008C1DBC2A83160313D6
:10058000111BE12A99228D229922831203138C01D7
:10059000913093008C1DCA2A83160313111BE12A84
:1005A000831603139115141CD32A83120313130803
:1005B000BA008316031391161116831203138C1DB0
:1005C000DF2A99229322F62208008316031318309B
:1005D0008700831603131413941783120313283010
:1005E0009400831603132930930008008316031325
:1005F0000030870083120313083094000800831230
:10060000031305110518022B8312031308001C2382
:10061000831203138510000000000000000000009A
:1006200000000000000000008514051C152B0000D0
:100630000000870105150800FF30AE00AE0B1E2B31
:100640000800061E212BFF221F3087000723AA0166
:10065000A901BB01BC010230BE000030B9006C240E
:1006600047240230BE000030B90083010630310259
:10067000031D5A2B8301FA302A02031D402B472BFE
:100680000618472BAA0A47251125061C3A2B472591
:1006900011258618552B830103012A020319792B92
:1006A000AA0347251125861C4B2B061A312B5724EC
:1006B000CE247B2B830192302A02031D602B692BF1
:1006C000472511258618692BAA0347251125861C65
:1006D0005A2B0618552B830103012A020319762B86
:1006E000AA0A47251125061C6B2B552B0630B10095
:1006F000422BB101642B061E7B2B0800061E7E2BAD
:10070000FF221F3087000723AA01A901BB01BC01FA
:10071000B1010330BE000030B9006C24472403301F
:10072000BE000030B900830106303102031DB82B32
:100730008301FA302A02031D9E2BA52B0618A52B38
:10074000AA0A1B251125061C982B1B251125861886
:10075000B32B830103012A020319D72BAA031B25FC
:100760001125861CA92B061A8F2B5724CE24D92B92
:10077000830192302A02031DBE2BC72B1B25112596
:100780008618C72BAA031B251125861CB82B061813
:10079000B32B830103012A020319D42BAA0A1B25B8
:1007A0001125061CC92BB32B0630B100A02BB101BB
:1007B000C22B061AD92B061EDB2B0800061EDE2BC9
:1007C000FF221F3087000723AA01A901BB01BC013A
:1007D000B1010030BE000030B9006C2447247325FD
:1007E000061EFF2B0F30B700061EFF2BFF30AD009B
:1007F0001D27AD0BF82BB70BF42B061AE42B061EA6
:10080000FF2B0800061E022CFF221F308700072343
:10081000FF221630870007233D14B801B901BE013D
:10082000FF2205300D2087000723FF223808022011
:1008300087000723FF2201300D2087000723AA012C
:10084000A901BB01BC01B101B9013808B9000030F0
:10085000BE006C2447243F1C73253F182C27FF2221
:100860000030172087000723061E432C2427B80AD0
:1008700008303802031D412CB801FF220B308700DD
:100880000723061A0F2C061E432C3D100800831266
:100890000313AA1B2A14AA13B1010310A90D0318EC
:1008A000532CB11431152908AA04A90108002A08FB
:1008B000A900AA018301A90C0318AA17A9130630DD
:1008C00083013102031DA9172A10AA102A11AA11A7
:1008D0002A12AA122A130800BF01E52299228722B0
:1008E0009922831203138C010310B90D9030B904BF
:1008F000390893008C1D7A2C83160313111BC72C07
:100900009922831203138C013E0893008C1D862CC0
:1009100083160313111BC72C99228D22992283124F
:1009200003138C013914390893008C1D952C831600
:100930000313111BC72C9922831203138C018316F6
:1009400003139115141CA22C831203131308A9007E
:100950008316031391121116831203138C1DAE2CF0
:100960009922831203138C01831603139115141C0F
:10097000B72C831203131308AA00831603139116CE
:100980001116831203138C1DC32C9922CB2C8312B6
:1009900003130130BF009322F6220800E5229922BA
:1009A00087229922831203138C010310B90D903012
:1009B000B90439088312031393008C1DDD2C8316B0
:1009C0000313111B0C2D9922831203138C013E0873
:1009D00093008C1DE92C83160313111B0C2D9922F7
:1009E000831203138C0183120313290893008C1DB7
:1009F000F72C83160313111B0C2D9922831203135A
:100A00008C01831203132A0893008C1D052D831675
:100A10000313111B0C2D99229322F622AA01A9017E
:100A200008000230B700FF30AD001D27AD0B152DBB
:100A3000B70B132D0800830103012A02031D222D89
:100A40000630B100A101A201A301A401A501A601E4
:100A5000A701A801AD01AB01AC01AF0183120313E3
:100A600005158514831203138701BB01BC012A08F5
:100A7000BB00063083013102031D402DFF26432DAC
:100A8000BB09BB0AFF266C26D826E6250800830191
:100A900003012A02031D4E2D0630B100A101A2015F
:100AA000A301A401A501A601A701A801AD01AB0105
:100AB000AC01AF01831203130515851483120313D0
:100AC0008701BB01BC012A08BB000630830131024B
:100AD000031D6C2DFF266F2DBB09BB0AFF266C265C
:100AE000D82627260800830103012A02031D7A2D38
:100AF0000630B100A101A201A301A401A501A60134
:100B0000A701A801AD01AB01AC01AF018312031332
:100B100005158514831203138701BB01BC012A0844
:100B2000BB00063083013102031D982DFF269B2D4B
:100B3000BB09BB0AFF266C26D8269F2508003D1856
:100B4000B82DFF22163087000723831203131130BC
:100B5000B700FF22831203130301013E8A00370806
:100B6000FE208700072383120313B70BA92D8A01E8
:100B7000FF2231080D2087000723FF2228080220CA
:100B800087000723FF222708022087000723FF2270
:100B90002608022087000723FF222C308700072326
:100BA000FF2225080220870007233D18E52DFF229C
:100BB00007300D2087000723FF2208300D20870013
:100BC0000723FF220B30870007230800FF2216307F
:100BD00087000723831203131130B700FF2203019C
:100BE0008312031337080000D820870007238312DD
:100BF0000313B70BEE2DFF2231080D2087000723CA
:100C0000FF222808022087000723FF22270802204E
:100C100087000723FF222608022087000723FF22E0
:100C20002C3087000723FF22250802208700072396
:100C3000FF2207300D2087000723FF2208300D20F8
:100C400087000723FF220B30870007230800FF22BD
:100C5000163087000723831203131130B700FF22D9
:100C60000301831203133708000000000000000096
:100C70000000EB208700072383120313B70B2F2EEE
:100C8000FF2231080D2087000723FF2228080220B9
:100C900087000723FF222708022087000723FF225F
:100CA0002608022087000723FF222C308700072315
:100CB000FF222508022087000723FF2207300D208E
:100CC00087000723FF2208300D2087000723FF221B
:100CD0000B308700072308003C08AC003B08AB0042
:100CE0008301AC0DAC0DAC0DAC0D8301AC0D031C40
:100CF0007F2E0230A4070430A2070830A107830129
:100D0000AC0D031C892E0130A4070230A207043069
:100D1000A1078301AC0D031C932E0530A3070130FE
:100D2000A2070230A1078301AC0D031C9D2E0230E7
:100D3000A3070530A2070630A1078301AB0D031CF2
:100D4000A72E0130A3070230A2070830A1078301B4
:100D5000AB0D031CAF2E0630A2070430A1078301A0
:100D6000AB0D031CB72E0330A2070230A10783018D
:100D7000AB0D031CBF2E0130A2070630A107830173
:100D8000AB0D031CC52E0830A1078301AB0D031C5E
:100D9000CB2E0430A1078301AB0D031CD12E0230F2
:100DA000A1078301AB0D031CD72E0130A10708005A
:100DB0000A30AF01A102AF0A0318DA2EA1072108F9
:100DC000A500AF032F08A2070A30AF01A202AF0AA5
:100DD0000318E62EA2072208A600AF032F08A307D8
:100DE0000A30AF01A302AF0A0318F22EA3072308AB
:100DF000A700AF032F08A4072408A8000800831247
:100E000003133B08B2000530B300B501B60108304A
:100E1000B400330883120313031083120313B60DB7
:100E2000B50DB20D0318B6070318B50AB40B0A2F97
:100E30003608BB003508BC000800FF30B000B00B1E
:100E40001C23031D1F2F0800FF30B000B00B292FFB
:100E50002B2F1C23262F0800FF2216308700072384
:100E6000831203130630B700FF22030100300D2068
:100E70008700072383120313B70B342FBF01080029
:00000001FF
